:100000003BC455C454C453C452C451C450C4B0C6F4
:100010004EC44DC44CC44BC44AC425C64AC647C48A
:1000200046C445C444C443C499C60204081001022E
:100030000201010201000002100408402002020136
:10004000010100000080805F8080808003000380C9
:1000500080147F147F14242A7F2A122313086462D9
:10006000364956205005038080801C224180804103
:10007000221C808022146B142208083E080850308D
:100080008080800808080880606080808060100898
:1000900004033E41413E80427F4080806251494698
:1000A0008022414936801814127F802745453980C7
:1000B0003C4A49318001710D03803649493680063A
:1000C00049291E803636808080563680808008140C
:1000D0002241801414141480412214088002510912
:1000E0000680324979413E7E09097E807F49493642
:1000F000803E414122807F41413E807F494941808D
:100100007F090901803E49493A807F08087F804184
:100110007F4180802040403F807F081463807F4083
:100120004040807F020C027F7F06187F803E414165
:100130003E807F090906803E41215E807F09196665
:1001400080264949328001017F01013F40403F80C4
:1001500007186018073F4038403F631408146303D2
:100160000478040361594543807F41418080030442
:1001700008106041417F8080020102808040404041
:100180004080030480808020545478807F48483029
:100190008038444428803844447F80385454488010
:1001A000047E05018048545438807F080870807AA6
:1001B0008080808020403A80807F08146280417F68
:1001C0004080807C047804787C040478803844443F
:1001D00038807C242418801824247C8078040480AF
:1001E000804854542480043F4444803C40407C80F8
:1001F0000C3040308C3C4030403C44281028444C6B
:1002000050503C8064544C448008364180807F804C
:100210008080804136088080080408100880808033
:1002200080801C2A4949221F047F4040201210125E
:1002300020102220221021545479807914147980BE
:10024000394444398039444439803D40407D803DC3
:1002500040403D807E25251A806C1A6F1A6C7D5AAD
:100260001E5A7D4E7B0F7B4E7C3A7E3A7C1C762E4E
:10027000761C1E347C341E0C1224120C081C3E7F8B
:10028000807F3E1C0880303F01627E303F028080CC
:100290001E3D777331607E7B7E60205F2380807E91
:1002A0007A7A7F80034579450310282428100814A2
:1002B0002A1408000000000036360836361E143CAA
:1002C000287844241D244442241D620108651C2210
:1002D0004146241D244C08443D44084C241D24461A
:1002E00001621D620142241D24427C4657467C7FE8
:1002F0002A2A7F802A7F417F2A0A0055000A304837
:100300004D33070629792906081C2A080808082AF7
:100310001C081608B107880776071B070B07E706B6
:10032000D206C7061C06BC05A2053D051405C3047C
:100330003B04D603A303840365033C031C222E2A3B
:100340001C1C222A2E1C1C222A2A1C1C222A3A1C73
:100350001C223A2A1C1C322A2A1C1C2A2A2A1C1C4F
:10036000262A2A1CFF7F7F7F7F7F1C1C1C1C1C08E9
:10037000080808080808080808000808080000001D
:10038000080000FF1C3E773E1C3E7763773E776394
:10039000416377634108416341081C0841081C3EE2
:1003A0001C08FF40404140404040434040404045E1
:1003B0004040404049404040405140404040214042
:1003C00040404051404040484148404840414048FA
:1003D0004040414040FF00027D000000017C0200DF
:1003E00000007A000000087204000008601000009D
:1003F00010680000002040100000002000000000F5
:1004000000000000000000000000000000000030BC
:100410000000007C543800793D243D797B3F163F35
:100420007B7E7C187C7E7C0810087C70081008702D
:1004300060082010601040002000FF0C40013006D2
:10044000300104401840061001600118400200030A
:10045000600108010C4042600650212420582013FE
:10046000581128100E680A101108680C1112086B38
:10047000081614096C0910100E680A10130C680C89
:100480001116086B081214096C0814100A68081376
:100490006F7717776F1009680A106F7717776F11EA
:1004A0000C680B101608690C1114096A1016100B51
:1004B0007C102C2016601340412C400C400360003F
:1004C0002801FF403C433C40407C437C40403C434F
:1004D0003C40407C437C40403C433C40407C437C2F
:1004E00040205E215E20106F106F1008770877089B
:1004F000047B047B04027502750201680168012017
:10050000502050204010200040200040004040007B
:10051000400000FF40404040404060504844446438
:10052000544C44446C546C44446C546C7C446C5542
:100530006E7C446E556E7C7C6E556E7CFF4040092F
:10054000010000454100000301404000050140401A
:1005500000094140000050410100006041010000DD
:1005600040510100000041510000000041490000DD
:1005700000414108000040450100000541400003E2
:1005800001404001050040400009014040001001C9
:1005900041400020414100004041410000404101F4
:1005A00000FF20505020003048483000060909065E
:1005B0000001020201000001010000FF0300000031
:1005C0000003000000000700000000060200000019
:1005D00005060000000C06000000080E0000000ADE
:1005E0000C040000080A0C000004180C000008109D
:1005F0001C00000014180800001014180000083037
:1006000018000010203800000028301000002028BA
:100610003000000000000000202830FF000007002C
:100620000000000E00000008080800101010000074
:100630002020200000404343000040464600004088
:10064000404C0C00404040181840404060600000A2
:100650000020204040406060000107444000020E3E
:1006600048400018084C403010184040602030408E
:100670004060273440407E303040407E313340403F
:100680007E323640407E303644407E30304C487EAC
:10069000303050587E303060705E101040507E30E8
:1006A0003060707C202040607C212744607C222EBA
:1006B00048607C38284C607C3B2B4C607C3E2E4C48
:1006C000607C3F2F4D60FF552A552A552A552A55E3
:1006D0002AFF10101010100810100F7010100808CA
:1006E000101010101010FF002620260000262026D3
:1006F00000002620260000262024000026202600B8
:1007000000262026001026202610FF00001C0000D6
:10071000003E223E007F4141417FFF01000000007A
:1007200002000100000400020000080104000110A2
:1007300002080002200411000441082200084210AF
:1007400044011045204802204A4050044154406072
:10075000084268416011447042602248704460451C
:10076000507048604A5070506054607060606860BB
:100770007060607060FF084428100804020408508C
:1007800030100804040201FF010000000002020111
:10079000000006090906000030484830002050508B
:1007A000200030484830000006090900000001021E
:1007B000FF785C6878717C38747C7A7850626278F3
:1007C0007C606170687A60307874707970526960AA
:1007D0007C687061506670782068716072507479BE
:1007E0007062687270306174617850707A743140F0
:1007F00068441068703460284A60586060703866D9
:100800001860707842195864702970703A78547082
:100810007051786A70FF142A49493E001C2A493EEB
:10082000003E493E087F2A1C0808221C0808081CB4
:100830000008080800080808080808080800080850
:100840000800000808000000080000000000000088
:10085000000C0000000C1200000C1224000C1224EA
:10086000120C1224120CFF321E120B070503020099
:1008700001020305080D150011241FBECFE5D1E0CC
:10088000DEBFCDBF10E0A0E6B0E0ECECFFE002C0C0
:1008900005900D92A836B107D9F711E0A8E6B0E0AF
:1008A00001C01D92A933B107E1F70DD38DC3A8CBC9
:1008B000CF93DF93CDB7DEB7C350CDBF8091340166
:1008C000853018F01092340103C08F5F809334019B
:1008D00020913401E0913301F0E0E559FF4FE20F40
:1008E000F11D308119821A821B8280E090E030FF76
:1008F00011C0FC01EF5CFF4F4491FC01E65DFF4F2E
:10090000E491A1E0B0E0AC0FBD1FA40FB11D4C916C
:100910004E2B4C93369501968730910541F780E038
:1009200090E0281789F0FC01E35CFF4F3491FC0153
:10093000E85CFF4FE491A1E0B0E0AC0FBD1FA30F56
:10094000B11D3C913E2B3C9301968530910549F7B2
:10095000998183E098278A812EE782278A838B8179
:100960002EE182278B838BB38C7F892B8BBB88B343
:1009700081789A81892B88BB82B3817E9B81892B68
:1009800082BBCD5FCDBFDF91CF910895F09135014E
:100990008F2F8F704F2F50E0BA0160717070E0910F
:1009A0003301F4FF02C0E81B01C0E80FA09136013B
:1009B0008E2F90E004962A2F30E082179307F4F0F0
:1009C00080913801882321F081508093380114C030
:1009D000809137018093380145FF05C080E18F2762
:1009E0008093350109C06115710521F0A550A093D0
:1009F000330102C01092330181E00895E093330186
:100A000080E008958F706370613019F04093380171
:100A100002C0109238016295682B609335014093B3
:100A200037010895109233011092360110926B0035
:100A300010926C0010926D0010926E0010926F0078
:100A40000895F0DF1092350110923701089520913A
:100A500036010BC0FC0134913F3F49F00196E22F73
:100A6000F0E0E559FF4F30832F5F283C98F3209347
:100A70003601089590913601983C40F4E92FF0E05A
:100A8000E559FF4F80839F5F9093360108958F3D16
:100A900049F0843C61F0863D79F08C3D79F0843EEC
:100AA00079F002C08AE811C0863F61F002C085E893
:100AB0000CC08C3F49F009C087E807C089E805C031
:100AC00084E803C086E801C088E88052813910F5C7
:100AD000E82FF0E0CF01880F991F880F991FEE5B78
:100AE000FF4FE80FF91F8091360195E001C0F90131
:100AF0009F012F5F3F4FE491E7FD0AC0883C30F42F
:100B0000A82FB0E0A559BF4FEC938F5F915079F7B4
:100B100080933601089583E08ABB8EE787BB8EE120
:100B200081BB8BB38C6F8BBB88B3816888BB82B36E
:100B3000816E82BB10BE85E083BF84E086BF87E202
:100B40008CBF89B7856089BF87E689B912B880E90B
:100B50008AB986E083B90895CF9320D2C82F83FF46
:100B600002C085E001C081E06C2F661F6627661F0A
:100B7000660FEC2FE295E770F0E0E159F74F4491F2
:100B800041DFC770EC2FF0E0E959F74FE491E093B3
:100B90006500CF910895EF92FF920F931F93CF932B
:100BA000DF930F92CDB7DEB77C01D6DF3BDF870145
:100BB0000E5F1F4FC7010196F1D1982F42C07801F7
:100BC0009E37A1F40894E11CF11CC801E7D18E37CF
:100BD00061F1E82FE154E53140F5F0E0EE0FFF1F41
:100BE000EE5EFC4F8591949132DF1FC09F3F81F4F0
:100BF0000894E11CF11CC801D1D107C03BDF87017B
:100C00000F5F1F4FC701CAD178018F3FB9F70DC0E1
:100C10009E3549F40894E11CF11CC801BFD1982FFE
:100C20008E3509F0915C892F32DF87010F5F1F4FEE
:100C3000C701B4D1982F882321F080E099831ADF6F
:100C40009981992309F0BBCFC801A8D1882311F459
:100C500000E010E0C8010F90DF91CF911F910F913C
:100C6000FF90EF9008951F920F920FB60F921124EC
:100C70002F933F934F935F936F937F938F939F93A4
:100C8000AF93BF93EF93FF9386B78C5F86BF10DE61
:100C9000FF91EF91BF91AF919F918F917F916F9154
:100CA0005F914F913F912F910F900FBE0F901F902A
:100CB00018951F920F920FB60F9211242F933F9306
:100CC0004F935F936F937F938F939F93AF93BF9354
:100CD000EF93FF938CB7895D8CBF8091660088236A
:100CE00021F081508093660005C08091650080935B
:100CF00066004CDE80B386FF08C08091640080FFF0
:100D00001CC0809164008E7712C08091640080FDC9
:100D100005C081E08093640084E60DC0809164008A
:100D2000813059F480916800882321F483E0809316
:100D3000640003C0815080936800FF91EF91BF91E0
:100D4000AF919F918F917F916F915F914F913F9163
:100D50002F910F900FBE0F901F9018951F920F921A
:100D60000FB60F9211240F900FBE0F901F90189581
:100D70001F920F920FB60F9211242F933F934F9310
:100D80005F936F937F938F939F93AF93BF93EF93F3
:100D9000FF936CB16B3119F486E080936900809108
:100DA0006900833009F441C0843028F4813089F02F
:100DB0008230E0F409C0853081F0853008F442C00B
:100DC000863009F06FC05FC0683409F06BC081E005
:100DD0004FC06C3409F066C04AC06D3009F462C07F
:100DE0006A3009F45FC082E0809369006E3511F4C7
:100DF00083E03EC0643221F410926A0084E038C07F
:100E000080916000909161009C012F5F3F4F309373
:100E10006100209360006D3011F06A3021F460E0D1
:100E2000C5D085E025C0C2D03DC0809160009091C2
:100E300061009C012F5F3F4F309361002093600061
:100E4000615C14C0962F9053913108F09750903107
:100E500090F080916000909161009C012F5F3F4F66
:100E6000309361002093600060916A009FD082E01F
:100E70008093690017C080916A008295807F890FF6
:100E800080936A000FC080E090E0909363008093AD
:100E900062009093610080936000C4DD81E8F7DD1B
:100EA00010926900FF91EF91BF91AF919F918F9147
:100EB0007F916F915F914F913F912F910F900FBE56
:100EC0000F901F90189527DEBCDD789481E8DFDD58
:100ED0008FEF94E3ACE081509040A040E1F700C078
:100EE0000000809162009091630055DE9093630052
:100EF00080936200C0E1D0E480916400882371F4A3
:100F0000809162009091630046DE9093630080932D
:100F10006200809164008068809364008091640026
:100F2000833051F77FDD82E8B2DD8FE79AE1A6E0FA
:100F300081509040A040E1F700C0000073DD8FEFCA
:100F400094E3ACE081509040A040E1F700C0000085
:100F5000CABFD5B9CBBF85B7806585BF85B780626D
:100F600085BF889585B78F7D85BF1BBE83E88FDDE4
:100F70008FE79AE1A6E081509040A040E1F700C0E1
:100F8000000080E090E007DE9093630080936200B1
:100F900080916400806880936400AECFE199FECFB9
:100FA0001FBA8EBBE09A99278DB30895262FE19939
:100FB000FECF1CBA1FBA8EBB2DBB0FB6F894E29AB7
:0C0FC000E19A0FBE01960895F894FFCF4F
:080FCC00000000008008010094
:00000001FF
